:1000000002021B1200E61200FF7F561201347F31FC
:100010001201347F2E1201347F351201347F3A12DF
:10002000026F1202968F08EF120249005B0300650F
:100030000800840A00760D00A511008B12007D18BF
:1000400000471B000000BF7F0A12026F7F2A1202C6
:100050006F1201468F0812012280C21202968F0889
:1000600012012280B87F101201227F201201347FFA
:100070001012012280A77F0212012280A07F0112AC
:10008000012280997FC01201228092D2B4D2B5D2CF
:10009000B3859008C2B3AF081201D17F027E00126F
:1000A00000CD02001DC2B4D2B5D2B3859008C2B350
:1000B000AF081201D17F027E001200CD02001DAFF9
:1000C0000812026FAF0812013402001D22EF4E60C9
:1000D000147D7D7C00ED1D70011CED4C70F7EF1F51
:1000E00070011E80E822C29FD29ED29DD29C75983C
:1000F0005053890F438920758DFDD28ED299227F6E
:10010000E87E031200CDC2B37F381201227F38127D
:1001100001227F381201227F061201227F0E120176
:100120002222C2B4C2B58F90D2B3C2B37FBE7E00CA
:1001300012020F22D2B4C2B58F90D2B3C2B37F05E0
:100140007E0012020F221202968F09D3E509648005
:1001500094E650F2C3E509648094E1400DAF0912C2
:10016000026F74A92509F509801DD3E509648094FF
:10017000B950D3C3E509648094B040CAAF091202F4
:100180006F74D02509F5091202968F0AD3E50A6427
:100190008094E650F2C3E50A648094E1400DAF0A12
:1001A00012026F74A9250AF50A801DD3E50A64803E
:1001B00094B950D3C3E50A648094B040CAAF0A1220
:1001C000026F74D0250AF50AE509C454F0250AFF28
:1001D00022AE07EE75F0101202272430FFEE75F004
:1001E00010120227AEF0EE2430F509D3EF648094AC
:1001F000B9400474272FFFD3E509648094B9400601
:1002000074272509F50912026FAF0912026F22EF58
:100210004E6007EF1F70011E80F522787FE4F6D84C
:10022000FD75810A020003C2D530F707B2D563F02D
:10023000FF05F030E70CB2D5F4048463F0FF05F05D
:1002400080018430D502F40422D083D082F8E49374
:100250007012740193700DA3A393F8740193F58247
:100260008883E4737402936860EFA3A3A380DFEF35
:10027000B40A07740D12027A740A309811A899B85A
:10028000130CC2983098FDA899C298B811F630990D
:10029000FDC299F599223098FDAF99C2987E00224F
:00000001FF
